:020000040000FA
:1000000000008A0103280730990083160313910129
:1000100070308F000F1D0A2800308100FF309500DE
:100020000830870083120313871101309300920177
:100030009115203084008001840A841F1B289717A3
:10004000203096000030F200403EF300403EF400C5
:10005000403EF5008316031387113C305720871567
:100060008312031356200000000000309500720830
:100070005220730852207408522075085220003014
:100080005220003052200030522000305220FF30E9
:1000900057200A30F107031C2A28F20AF30AF40A4F
:1000A000F50A2A288C1C522895008C100800F000B4
:0600B000F00B58280800C7
:02400E00E43399
:00000001FF
